:020000040000FA
:10000000682C0020F9020000010300000303000037
:1000100005030000070300000903000000000000C2
:100020000000000000000000000000000B030000C2
:100030000D030000000000000F030000110300008A
:100040001303000029060000290B00001303000021
:100050001303000013030000F50300001303000066
:10006000C50A00001303000013030000130300007F
:100070001303000013030000130300001303000028
:1000800013030000B906000013030000130300006F
:10009000DD060000E106000013030000130300006A
:1000A00013030000130300001303000013030000F8
:1000B0001303000013030000000000000000000014
:1000C00013030000130300001303000013030000D8
:1000D00013030000130300001303000000000000DE
:1000E0000000000000000000000000000000000010
:1000F0000000000000000000000000000000000000
:1001000000000000000000000000000000000000EF
:1001100000000000000000000000000000000000DF
:1001200000000000000000000000000000000000CF
:1001300000000000000000000000000000000000BF
:1001400000000000000000000000000000000000AF
:10015000000000000000000000000000000000009F
:10016000000000000000000000000000000000008F
:10017000000000000000000000000000000000007F
:10018000000000000000000000000000000000006F
:10019000000000000000000000000000000000005F
:1001A000000000000000000000000000000000004F
:1001B000000000000000000000000000000000003F
:1001C000000000000000000000000000000000002F
:1001D000000000000000000000000000000000001F
:1001E000000000000000000000000000000000000F
:1001F00000000000000000000000000000000000FF
:10020000DFF80CD000F0C6F800480047552B00007E
:10021000682C002030B4044654E8000F0D4644E832
:100220000053002BF8D1156030BC704730B4044641
:1002300054E8000F40EA010544E80053002BF7D1D1
:10024000156030BC704730B4044654E8000F00EA33
:10025000010544E80053002BF7D1156030BC70470E
:1002600030B4044654E8000F80EA010544E8005326
:10027000002BF7D1156030BC704730B4044654E809
:10028000000F00EB010544E80053002BF7D1156087
:1002900030BC704730B4044654E8000FA0EB0105B1
:1002A00044E80053002BF7D1156030BC704770B4A0
:1002B00004464FF0000054E8006F0D68AE4207BFDF
:1002C00044E80023012044E800630E60002B1CBFBB
:1002D0000020F0E770BC704730B4044654E8000FCB
:1002E00088422CBF451A054644E80053002BF5D13F
:1002F000156030BC7047000006488047064800473C
:10030000FEE7FEE7FEE7FEE7FEE7FEE7FEE7FEE7C5
:10031000FEE7FEE7550700000102000000487047B5
:100320003C74000040EA01039B0703D009E008C9C0
:10033000121F08C0042AFAD203E011F8013B00F8AA
:10034000013B521EF9D27047D2B201E000F8012BF6
:10035000491EFBD270470022F6E710B513460A4645
:1003600004461946FFF7F0FF204610BD421C10F866
:10037000011B0029FBD1801A704730B504460020CC
:10038000034600E05B1C934203D2E05CCD5C401B63
:10039000F8D030BD064C074D06E0E06840F00103A0
:1003A00094E8070098471034AC42F6D3FFF72CFFCF
:1003B000DC740000FC74000030B58C1810F8012BC0
:1003C00012F00F0301D110F8013B120906D110F809
:1003D000012B03E010F8015B01F8015B5B1EF9D112
:1003E00001E001F8013B521EFBD1A142E6D30020FF
:1003F00030BD00002DE9F04700268AB0DFF85091AB
:10040000B0464FF48075012437460696284603F01F
:10041000DDFA38B1D9F80403204203D0284603F0AE
:10042000CBFA26432D1D64007F1CADB2082FEDD3FF
:100430004FF4BE74204603F0C9FA48B1204603F0D9
:10044000BBFA46F0004606AA0121002003F0A0FAFC
:10045000404D16F0FF0F15D00127002437420DD074
:1004600009EB8401D1F81005D1F81015C0F3042070
:1004700055F82420C1F3014102B190477F00641C6C
:10048000082CEBD3002E5FDA4FF0FF30CDF8108050
:1004900054E0281910F8507F90F9000027F0C008A8
:1004A000401C3BD007A9404602F0B8FD10B34FEA0C
:1004B0009719404600F0ECFC55F820701FB1B9F1D7
:1004C000030F03D006E0B9F1030F27D104A940467A
:1004D00002F0ACFD4FF0A04101EB8800D0F800071E
:1004E00006A9C0F3014A404602F098FD18B1BAF1DE
:1004F000020F03D012E0BAF1030F0FD1B9F1030FCD
:1005000008D1BAF1020F1DD00221404603F024FAAF
:10051000761CF6B217B149464046B847641C042C15
:10052000B7D3002E10D06A460121002003F030FA24
:1005300006990098884207D0069004980026344611
:100540000790A6E70321E0E70AB0BDE8F0870000C6
:10055000006000408401002000F01F020121914052
:100560004009800000F1E020C0F88012704700F0E0
:100570001F02012191404009800000F1E020C0F8F5
:100580008012704700F01F02012191404009800055
:1005900000F1E020C0F88012704700F01F02012136
:1005A00091404009800000F1E020C0F880127047BF
:1005B00000F01F02012191404009800000F1E0207D
:1005C000C0F88011704700F01F02012191404009DE
:1005D000800000F1E020C0F80011704700F01F0219
:1005E000012191404009800000F1E020C0F8001195
:1005F000704700F01F02012191404009800000F186
:10060000E020C0F8001270474907090E002806DAFA
:1006100000F00F0000F1E02080F8141D704700F199
:10062000E02080F80014704770B5204D28696C7880
:10063000401C2861687D10B11D4802F07FFC2878BD
:1006400003281AD11B48D0F80C01B0B1012C04D0FA
:10065000022C0AD01648123023E02869032816D04D
:100660001348083002F06AFC11E02869022812D011
:100670000F480D3002F062FC0DE0032C0FD2012C6C
:1006800005D0022C07D0BDE8704004F05DBCBDE889
:10069000704004F085BCBDE8704004F097BE04488B
:1006A0002830BDE8704002F049BC00001809002065
:1006B00038030A000010004007480021C0F840112C
:1006C000C0F84411C0F84811C0F84C11C0F800112E
:1006D000C0F8041106F0FABB0010014006F068BB38
:1006E00030B51B4C85B00025012080F31088D4F86C
:1006F000D40038B3D4F8D00000EB800004EB8000C5
:1007000001798DF800108168C26803694069CDE9FC
:100710000330CDE90112D4F8D400401EC4F8D4004F
:10072000D4F8D000401CC4F8D000D4F8D0000A2877
:1007300001D3C4F8D050002080F3108821686846A7
:100740008847D1E7002080F3108805B030BD000055
:1007500034090020F0B5B5480023021D0178101DB2
:1007600001254FF0805406290BD11678360708D1A1
:100770000678C6F30316032E06D0042E04D0052EE9
:1007800002D0062907D00EE0B4F82463A84FC6F3C0
:1007900004263E6002E01678360704D10678C6F3D8
:1007A0000316032E02D0062904D00FE0A24FA14E5B
:1007B0007E670EE01678360708D10678C6F3031672
:1007C000032E06D0042E04D0052E02D0062907D011
:1007D0000EE0D4F84462994FC6F342363E6002E020
:1007E0001678360704D10678C6F30316032E02D016
:1007F000062906D011E0924E376827F080773760DF
:100800000EE01678360708D10678C6F30316032ED5
:1008100006D0042E04D0052E02D006290AD011E0FD
:100820004FF08046C6F80C31C6F81031834E361FA3
:10083000336002E01678360704D10678C6F3031653
:10084000032E02D0062905D00CE07C4F0326643726
:100850003E600AE01678360704D10678C6F3031620
:10086000032E02D006290DD014E0764F05263E60F7
:10087000744E78363560734E083633603F263F1D20
:100880003E6002E01678360704D10678C6F30316F8
:10089000052E02D0062957D062E06B4E36686B4FAA
:1008A0003E60694E361D36683F1D3E60664E083616
:1008B00036683F1D3E60644E0C3636683F1D3E6014
:1008C000614E103636683F1D3E605F4E1436366806
:1008D0003F1D3E605C4E183636685C4F20373E60E8
:1008E000594E1C3636683F1D3E60574E20363668DE
:1008F0003F1D3E60544E243636683F1D3E60524ECA
:10090000283636683F1D3E604F4E2C3636683F1DF8
:100910003E604D4E303636684C4F40373E604A4E52
:10092000343636683F1D3E60474E383636683F1DC8
:100930003E60454E3C3636683F1D3E60424E403676
:1009400036683F1D3E6002E01678360708D106780B
:10095000C6F30316032E06D0042E04D0052E02D0B3
:10096000062907D019E0D4F85812394A01F04F018E
:10097000116002E0117809070FD10078C0F303106D
:10098000032803D0042801D0052806D13148016886
:10099000C90702D06FF001010160D4F830010628C8
:1009A00008D1D4F83401062804D12B48016841F459
:1009B0008061016022487438016841F4700101606F
:1009C000BFF34F8FBFF36F8F4FF01021D1F80002AC
:1009D000002803DBD1F80402002822DA1F4A156040
:1009E0001F480468002CFCD01524C1F8004205689B
:1009F000002DFCD0C1F8044201680029FCD013602E
:100A000001680029FCD0BFF34F8F0D48F038016812
:100A1000144A01F4E06111430160BFF34F8F00BF3E
:100A2000FDE7124910480860F0BD0000E00F00F03B
:100A3000403501400DF0ADBA00C007403C05004014
:100A4000FCED00E0105600400404001020C50040FA
:100A5000E40E0040000400403C17004004E5014063
:100A600000E401400400FA050090D003C800002013
:100A7000124A10B50021104B126809E053F82140CA
:100A8000844203D10E4802F059FA13E0491CC9B25E
:100A90009142F3D3084A002112F1180201EB01132D
:100AA00002EB4303834201D1012010BD491CC9B2AE
:100AB0000629F3D3002010BD800B00203801002050
:100AC000EC00030070B5144E4FF48030C6F80803F4
:100AD0000025C6F84051114C606810B9104802F06A
:100AE0002DFAA57062680123656073640D48016882
:100AF000001F00681430B1F5804F04D2B0F5404FAC
:100B000001D9637005E0814201D3012000E000209B
:100B10006070BDE870401047008000401001002068
:100B2000E5000400448500400148006800470000DB
:100B30001800002002E008C8121F08C1002AFAD1DC
:100B400070477047002001E001C1121F002AFBD14D
:100B50007047000072B605F0C1F900BF05F014F847
:100B60000028FBD1104C0121208801EB00400FA18F
:100B700005F016F910480068C00700D000BE2088B4
:100B8000022101EB00400DA105F00AF9BFF34F8FE0
:100B90000948E43801680D4A01F4E061114301603D
:100BA000BFF34F8F00BFFDE7500100204661746125
:100BB0006C206572726F7200F0ED00E0537973740F
:100BC000656D207265736574000000000400FA050D
:100BD0000EB500210091CDE901106A4644F20100F2
:100BE000FFF7B8FF0EBD00F003B800F009B8000031
:100BF00072B602480168491C016070473400002049
:100C000003490868401E086000D162B670470000C2
:100C1000340000202DE9F041064608680C46411CCE
:100C20004FF0A0474FF0010506D005FA00F1C7F8D4
:100C30000815206802F07CFE6068411C02D000218B
:100C400002F064FE3168A069C1F82405607D227D50
:100C500031681043C1F86C05D4E900123068C0F85F
:100C60001425C0F80C15207D012815D1A068411C61
:100C700002D0002102F04AFEE068411C05D0854008
:100C8000C7F80855E06802F053FED4E90212306854
:100C9000C0F80825C0F81015BDE8F0812DE9F04135
:100CA000064608680C46411C4FF0A0474FF001056E
:100CB00006D005FA00F1C7F80815206802F042FED8
:100CC0006068411C02D0002102F029FE3168A06951
:100CD000C1F82405607D217D32680843C2F86C05A7
:100CE000D4E900123068C0F80C15C0F81425207D36
:100CF000012815D1A068411C02D0002102F00FFE8E
:100D0000E068411C05D08540C7F80855E06802F04E
:100D100019FED4E902123068C0F80825C0F8101591
:100D2000BDE8F0810649095C4FF0A040D0F81005FD
:100D3000C84010F0010000D0012080F00100704791
:100D40000C7300002DE9FC410646C0074FF000057A
:100D50000ED0104F00240122385D0095002311466B
:100D6000019502F08BFD641C042CF4D300F01CF8F8
:100D7000B0070DD5074E0024361D0022305D032339
:100D800000951146019502F079FD641C042CF4D302
:100D9000BDE8FC81087300000249085C012102F0F3
:100DA000ECBD00000873000010B500242046FFF7DA
:100DB000F3FF641C042CF9D310BD042801D2FFF703
:100DC000B1BF0020704710B50024FFF7BBFF2046DD
:100DD00010BD00002DE9F0470546861C90460F46E1
:100DE0004FF001090020FFF7FEFE1B4C2068386021
:100DF000D4E90001401AA16804F21C47081A0EE069
:100E00000121384602F0A2F801F056FE01463846AC
:100E100002F09CF8D4E90001401AA168081A401CAD
:100E20008642EDD8B8F1000F03D0052065F3891094
:100E300002E0062065F39F50A2682168114004EB90
:100E40008101C8602068304420600020FFF7CDFE9B
:100E50004846BDE8F08700003C04002030B48268BA
:100E60000468531C8360A154D0E901128A4202D362
:100E700030BC02F00ABC30BC70470000034803C815
:100E8000814201D101207047002070473C040020BE
:100E90000249084490F930007047000084010020A6
:100EA0002DE9F05F26484168F1B3DFF898B00E688D
:100EB0008146DBF8004087688078E11B21F07F45A0
:100EC000ED1CB0B9DFF880804FF48030C8F84403DF
:100ED000C8F804031120FFF73FFB1120FFF773FB55
:100EE0004FF0010AC8F800A02F2005F0ABFB89F8ED
:100EF00002A0B54200D23546124BE8193C3320F02F
:100F00007F401860DBF800105A46091B21F07F4132
:100F1000001B20F07F40C91C81420FD91068186067
:100F20002F2005F08FFB00E004E0BDE8F05F11200A
:100F3000FFF75FBBBDE8F05F05F086BEBDE8F09F40
:100F400020000020041501400010014010B50021D0
:100F5000024802F006F880F3100010BD5808002087
:100F60000E4910B50A784C780023A24212D0521CC8
:100F7000D2B20A70022A00D10B70084A0B780C32E8
:100F800052F8232002608868104420F07F40886077
:100F9000012010BD0360002010BD000020000020D3
:100FA00002490A8802808978817070476473000062
:100FB000002207E010F8013BFF2B01D00020704712
:100FC000521CD2B28A42F5D30120704770B50C464C
:100FD00005460D2910D801F0EBF808B1012070BDCD
:100FE0000648007840B901F01FFA28B1214628468A
:100FF000BDE8704001F0DCB8002070BDB2000020F8
:10100000FFFFFFFFFFFFFFFFFFFFFFFFFFFFFFFFF0
:10101000FFFFFFFFFFFFFFFFFFFFFFFFFFFFFFFFE0
:10102000FFFFFFFFFFFFFFFFFFFFFFFFFFFFFFFFD0
:10103000FFFFFFFFFFFFFFFFFFFFFFFFFFFFFFFFC0
:102000002DE9F0418AB020270026099701F0D6FD7E
:10201000054601F0EBFD804601F04EFFC82001F0BF
:10202000D9FE052001F00EFF002001F097FD01F020
:1020300045FD00208DF8200004460022012108A85B
:1020400000F028FB30B1002001F044FF641CE4B232
:10205000642CF2D3C82000F0EFF801208DF82000A6
:102060000146002208A800F015FB08B31E480078BE
:10207000F0B1002001F0A4FD00281DDD09AA694689
:102080000020099701F034FDB0B19DF80000082848
:1020900012D11548DDF801100C38C0F803100DF10D
:1020A000010000F059FB002000F000FA012603E0D7
:1020B0004FF4967000F0C0F84FF4AF7000F0BCF829
:1020C00001F0FAFE002001F049FD002001F056FD6C
:1020D000284601F07FFE404601F0B4FE01F0EEFC20
:1020E0000AB03046BDE8F081BE000020F0B50746DA
:1020F000204889B0154600780E4698B1012814D0C2
:10210000022834D110221C4904A8FEF70BF91B4900
:102110000D2204A8FEF706F90024164A6846521C50
:1021200021460DE010221449F3E71022124904A8B9
:10213000FEF7F8F804A800F0C5F8EDE7052C02D288
:10214000135D035500E00155641CE4B2102CF5D377
:1021500001F07EF804A801F08DF86946084601F008
:102160004DF82B466A463146384600F055FB09B01B
:10217000F0BD0000AC000020677300008008002064
:102180000149087070470000AC00002001460D2294
:102190000148FEF7C7B80000800800200349026824
:1021A000C1F801200079487170470000AC000020A0
:1021B000F0B50746081D89B0C6B206208DF810009C
:1021C00004AC0D46601CFEF7EBFE2A463946201D86
:1021D000FEF7A8F8174D287808B1002000E002208B
:1021E000FFF7CEFF701EC2B2611C601CFFF77EFFBE
:1021F00001200090002301AA314604A800F060FAF3
:1022000018B99DF804000B2802D0002009B0F0BDD9
:1022100001AC0322A01DA11DFFF768FFA01D00F067
:10222000EFFA0028F2D0287810B9601CFFF7B6FF4B
:102230000120EBE7B200002010B5044601F0D4FC09
:102240006043400004D00349BDE8104080010847C6
:1022500010BD000081730000014803F081BF000041
:1022600000100000F0B54E23B3FBF2F5022303701B
:102270004F23841804F8013C81B10123541E0BE064
:1022800003F003068E5DB6FBF5F705FB176605FB4D
:102290000366C6545B1CDBB2A342F1DB01210DE0F7
:1022A0004318445C13F8013CE31ADBB2052B03D25C
:1022B000C3F1050323444354491CC9B29142EFD3EF
:1022C000F0BD00000349D1F807200260C97A01710E
:1022D00070470000B2000020F0B52F4D87B00026F7
:1022E0002878012701ACB0B103208DF80400601CF0
:1022F000FEF756FE0020FFF743FF0322611C601C1F
:10230000FFF7F4FE002303AA042101A8009700F0C0
:10231000D7F9A0B117E002208DF804000521601C58
:1023200000F086F90122062101A800F0B3F950B1AE
:10233000601CFFF733FF2F70002007B0F0BD9DF841
:102340000C00092802D02E700320F6E703AC092206
:10235000601C611CFFF7CAFE601C00F051FAC0B19E
:102360009DF8100020B1012805D0022800D12E7060
:102370009DF81000E1E7601D00F076F90D21074897
:1023800000F056F90548FFF701FF012000F08EF834
:10239000EDE72E700220D0E7B20000208D0800206B
:1023A00041F6FF700078FF2801D00120704700201F
:1023B000704740F6817041F27E01095CFF2905D02B
:1023C0000F20B0EB111F07D008097047401E00B264
:1023D0000028F0DA0E20704701F00F00704700006F
:1023E0003EB5104C00202070FFF7DAFF98B94FF48B
:1023F000805090F87E00FF280DD0FFF7DAFF0146ED
:102400000E2808D2684600F046F80098C4F8030089
:1024100001A800F029F9BDE83E400248C01C00F0C8
:102420009BB90000B200002010B58AB004208DF8DE
:102430000400012001460090002306AA01A800F034
:102440003FF930BB9DF818000A2822D10DF1190080
:10245000FFF7A4FE05208DF8040001AC601CFEF718
:102460009FFD0D21201D00F0E3F8201DFFF78EFEDB
:102470000120FFF785FE1022611C601CFFF736FE6D
:102480000122112101A800F005F910B101200AB0C4
:1024900010BD0020FBE701EBC10101F580510A6886
:1024A00002604A684260097A017270472DE9FE4372
:1024B00000265E4FB046344600285ED00025E9462F
:1024C00029466846FFF7E7FF58490422C91C6846B9
:1024D000FDF753FF38B955490522C91D09F104001C
:1024E000FDF74BFF80B16D1CEDB20E2DE8D300253A
:1024F00029466846FFF7CFFF4C490422C91C6846AD
:10250000FDF73BFF10B10CE02C4632E0052109F14C
:102510000400FEF74DFD20B1D7F807000190F87ACE
:1025200013E06D1CEDB20E2DE2D30025294668465E
:10253000FFF7B1FF09216846FEF73AFD48B157F8A9
:10254000030F009078680190387A8DF808002C46C7
:1025500031E06D1CEDB20E2DE8D3B8F1000F07D0BD
:1025600004EBC4006946092200F5805003F032FEF6
:102570003EB3FFF715FF28B356E000242146684616
:10258000FFF789FF29490422C91C6846FDF7F5FEBB
:102590000028EED0641CE4B20E2CEFD300242146B8
:1025A0006846FFF778FF04216846FEF701FD20B179
:1025B000D7F8030000900126D2E7641CE4B20E2C89
:1025C000EDD331E0FFF7F5FEA0422DD00E2C2BD03D
:1025D0004FF48051002040F681720F2591F87E1053
:1025E000531C04E041F27E019042095C0DD0CE43C1
:1025F000360706D0B5EB111F0AD164F31F11C9B21B
:102600000AE001F0F001214306E044F0E00103E0BC
:10261000401C00B29842E5DB41F27E02104403F018
:10262000B7FD0120BDE8FE830020FBE7B2000020DB
:10263000F0B50B4B0025C3F8005101241C602A465D
:10264000084E09E0D3F80071002FFBD0376887549B
:10265000C3F80051521CD2B28A42F3D35C60F0BD81
:1026600000D0004008D5004003490268C1F80720A7
:102670000079C87270470000B200002010B504460F
:1026800001F0F4F900E030BF01F0A8FAB0EB440F1C
:10269000F9D310BD10B5094C134600226270A27028
:1026A0000A460146184601F099F908B910BD30BF35
:1026B00060780028FBD0A07810BD0000B200002098
:1026C0002DE9FC4780460A200A9D009016460F46D9
:1026D000284601F0FFFB012401F0E2F901F0ECFAD9
:1026E0000028FBD101F078FA81461E2001F08AFB18
:1026F00001F0E4F92A4639464046FFF7CBFFE0B146
:102700000224284601F0E6FB07208DF804000A2089
:10271000FFF7B4FF2A46012101A8FFF7BBFF60B114
:10272000284601F04DFA40B1202000906A4631461B
:10273000284601F0DDF900B1002401F0B1F900BF35
:1027400001F0BAFA0028FBD1484601F05BFB01F02A
:10275000B5F92046BDE8FC872DE9FF41054601F0AB
:10276000ABFA264C0646EDB328786978EA7800EB98
:102770000120A978090401EB0261471801F09CFBD4
:10278000204601F0B5FA50B10021084601F09CFA4C
:1027900028B1384601F0BCFA08B1012402E0012456
:1027A00007E037B12146084601F08EFA08B101274B
:1027B00000E00027641CE4B2082CF2D301F0F2F927
:1027C0000446C2B229466846FFF74CFD87B1214650
:1027D000684601F0ADFA58B10120002E05D001F095
:1027E0006DF900E007E030B1012004B0BDE8F081F0
:1027F0000020002EF9D00020F7E700000406080AA8
:1028000010B503220349FDF7B8FD08B1002010BD43
:10281000012010BD6473000070B5002409E000BF02
:1028200011F8015B12F8016B7540641C00F8015B44
:10283000E4B29C42F4D370BD0278521C027002785C
:102840008A4201D300210170704700002DE9FC5F2E
:102850000E008346DDE90C47C6F10000984692461B
:10286000814600D40846012503E000BF90FBFAF042
:102870006D1C5045FADAA84500D9454624B1002E12
:1028800001DB780700D5641EB80702D5B8F1000F48
:102890000AD0F80708D13CB1A54205D220215846FC
:1028A000641EFEF7DBFAF6E7002E02DA4E462D2113
:1028B00002E0780703D52B215846FEF7CFFA07F040
:1028C000030002280BD1B8F1000F08D13CB1A5429A
:1028D00005D230215846641EFEF7C0FAF6E7CDE96E
:1028E0000047434652463146584604F0B3FCBDE823
:1028F000FC9F000070B50D46044600684FF48871D7
:1029000003F09AFE4FF49071206803F095FE4FF4A7
:102910009271206803F090FE4FF4A271206803F0DA
:102920008BFE20681249C0F8041320686907000B69
:1029300040B2090E002806DA00F00F0000F1E02096
:1029400080F8141D03E000F1E02080F800142068F6
:102950000121000B40B200F01F02914040098000AD
:1029600000F1E020C0F88012C0F8001170BD000036
:1029700010030200024600201268930702D053079A
:1029800002D47047500714D502F00300012802D08A
:1029900002280CD105E0C2F383100B68801C184498
:1029A00004E00223086803EB9252104408600120FF
:1029B0007047086800EB9253C2F38910401CEEE7A1
:1029C0002DE9F047394E002780463D46DFF8E0907C
:1029D000D6F804A057E003D00446D0F81C8035E0B8
:1029E00099F8002002EB4201521CD2B289F8002073
:1029F00009EBC10199F80230091D9A4201D189F809
:102A0000005048680A780446012A12D0022A02D0EF
:102A1000032A3BD108E004F029FA00B1012725740C
:102A200034E00574C06900E070680028F9D1706076
:102A30002CE0207C50BB88686060C868A060086992
:102A4000E0604869A061F07800B165606268B168D3
:102A5000184B501A20F07F40984202D2A1680844D7
:102A600006E0881AA16820F07F40814202D9081A46
:102A7000206000E0256065600120A560207420468C
:102A8000E56104F0D5F9B8F10000A4D199F800107F
:102A900099F801008142A3D117B97168514502D05C
:102AA0000120BDE8F0870020FBE7000020000020A7
:102AB00030020020FFFF7F002DE9FF410026234860
:102AC00000F041FA2148001F074600F03CFA204C74
:102AD00060680090A56800E000986946284004EB13
:102AE00080000C30FFF746FF0028F5D101AA0099BD
:102AF00001EA050304EB8303491CDB6842F820303C
:102B0000401C00910228F2D3019800F00300012834
:102B10000BD0022810D10198032101EB90500099AD
:102B2000BDF80A6001EB900005E00198BDF80A606D
:102B3000C0F3831008440090384600F001FA08B151
:102B40000098606004B03046BDE8F0815408002071
:102B50003C0400204FF0000988B04E464FF00408B6
:102B600049460220FEF72FF908B1FEF731F84FF47D
:102B70000041002003F06EF908B1FEF729F802F0D9
:102B8000F5FF002001F054F828B901F011F800F524
:102B90000340FEF71DF84B2001F01CF94FF4FC70C8
:102BA00001F040F928B901F003F800F50340FEF701
:102BB0000FF8FFF751FBFFF713FC00F07FFF28B978
:102BC00000F0F6FF00F50340FEF702F8DFF8C4A0BE
:102BD0000321BAF8000001EB00402FA103F0E0F858
:102BE0005FF0010502F0D0FF0028FBD100273C4632
:102BF0002046FEF7E2F818B105FA04F03843C7B2F0
:102C0000641C042CF4D3F8438DF8000026B10D2188
:102C10006846FEF7DBF911E001F074F901F078F98C
:102C200011226946022000F0D9FE08B908E030BF41
:102C300001F074F90028FAD001F076F981460BE032
:102C4000BAF8000022A105EB004003F0A9F800BF8C
:102C500002F09AFF0028FBD186F00106B9F1000FBF
:102C600010D1BAF800001EA105EB004003F098F85F
:102C700002F08AFF0028FBD1FFF7C2F910B1FFF77D
:102C80002BFB8046B8F1000FB0D1FFF725FB804643
:102C9000ACE700005001002047617A656C6C20644D
:102CA000796E616D69632070616972696E67206514
:102CB00078616D706C6520737461727465642E2028
:102CC000446576696365206D6F64652E00000000C1
:102CD0005458206669666F206572726F722000001A
:102CE00047617A656C6C653A207472616E736D69C8
:102CF0007373696F6E206661696C65640000000023
:102D00002DE9F047C7880446181D16468946B0FBD2
:102D1000F7F1B0FBF7F207FB12009A193A44D21C04
:102D2000B2FBF7F2DDF820A001E02468491E00297B
:102D3000FBD13D1A8846B54216D818E0BAF1000F0B
:102D400005D0211809EB08002A46091D04E020449B
:102D500009EB08012A46001DFDF7E4FA002024686B
:102D6000761BA844B74201D9354600E03D46002E07
:102D7000E4D1BDE8F087000030B5024659B103F058
:102D800095F80021074C09E004EB810315685B8886
:102D9000AB4202D11160002030BD491C8142F3D307
:102DA000052030BD3C0100202DE9F0415C4903784D
:102DB0000446D1E903020025082B77D2DFE803F0AF
:102DC000042B4877726E8795217C914208D238B1E6
:102DD00000EB81018A6C521C8A640168491C016005
:102DE000A17B2E4661F307062189677B61F31F46AD
:102DF0006189606861F30F05217B61F31745E17B11
:102E000061F31F6501F0AEFC2A4631463846BDE845
:102E1000F04100F03BBE4869407D10B9414800F0E8
:102E20008DF82F46218965F3070761F31F476189F4
:102E3000267B61F30F05617B606861F31F6501F01C
:102E400091FC2A4639463046BDE8F04100F014BEF8
:102E5000217B914208D238B100EB81018A6C521C6F
:102E60008A640168491C0160A07A217A60F3070531
:102E700061F30F25E17A667A676861F3174538B127
:102E80001FB92848263000F059F8384601F06AFC8E
:102E900029463046BDE8F04100F0C9BEBDE8F0412A
:102EA00000F00ABE00F00EFFBDE8F08131E01E48E0
:102EB0004168491C416001780029F5D0816811B151
:102EC000491E8160F0E7BDE8F04100F0E9BDA3795B
:102ED000934208D238B100EB830293685B1C936085
:102EE0004268521C42608A680CE0A379934208D27F
:102EF00038B100EB830293685B1C93604268521CFC
:102F000042604A68002ACFD061792079BDE8F0415B
:102F10001047BDE8F04103487F3000F00FB80000D3
:102F2000CC0000203D0405009C08002002490F222F
:102F30000A70886170470000CC000020FFF7F6BFE0
:102F4000002100F009B8012100F010B808B56A4668
:102F5000FDF793F9009808BD08B56A46FDF773F9C7
:102F600008BD08B56A46FDF755F908BD08B56A46BB
:102F7000FDF75CF9009808BD08B56A46FDF78AF9C7
:102F8000009808BD70B5044600252846FDF72BFEC5
:102F900021686268086890420ED9401E0860017876
:102FA000A38AE26801FB0325227A2168101AC0B2C5
:102FB0000A79824200D208710020FDF716FE2846E9
:102FC00070BD70B505460C460020FDF70CFEE868A4
:102FD000A98A201AB0FBF1F12A681068431C13601B
:102FE0000170BDE870400020FDF7FFBD10B530B1A5
:102FF000017A42680368891AC9B21A6006E00E2095
:1030000010BD03681A68541C1C601170491EC9B2B7
:10301000F7D2006800210171084610BDC20800F017
:1030200007030120895C98400840704710B5C2082A
:1030300000F00703885C01249C402043885410BDA5
:1030400070B5074C251F206829684968884202D35B
:103050000448FFF773FF286821688068405C70BDF2
:10306000080100204400010001480068704700008A
:103070000801002010B50446054800684068A042D9
:1030800002D80448FFF75AFF0148001D046010BD34
:10309000040100204C000100014840687047000016
:1030A0000801002010B50446054800680068A042E9
:1030B00002D80448FFF742FF0148001D446010BDDC
:1030C000040100205800010010B5040002D1054899
:1030D000FFF734FF044800210460001D01604160D7
:1030E00010BD000027000100040100200948021F54
:1030F0004168491C416012681368994208D3002353
:1031000043600168491C01605268914200D303602A
:103110007047000008010020002839D0401E00BF81
:1031200000BF00BF00BF00BF00BF00BF00BF00BFA7
:1031300000BF00BF00BF00BF00BF00BF00BF00BF97
:1031400000BF00BF00BF00BF00BF00BF00BF00BF87
:1031500000BF00BF00BF00BF00BF00BF00BF00BF77
:1031600000BF00BF00BF00BF00BF00BF00BF00BF67
:1031700000BF00BF00BF00BF00BF00BF00BF00BF57
:1031800000BF00BF00BF00BF00BF00BF00BFC5D170
:1031900070470000F0B505460478154889B016461A
:1031A00040F82420124A0869121DA2F1080742F8CB
:1031B0002400487F385520226846FDF7B3F8049470
:1031C0002878385C48B10EB10A4A00E0002269460E
:1031D000281D03F09FFB09B0F0BD0EB1064A00E0C8
:1031E0000022694605F10C0003F066FAF3E70000DF
:1031F00004000020317100007D6F000070B5124D99
:1032000006464FF080746868814202D01022FDF7B4
:1032100089F80E490020C1F8000101220A6001E08E
:10322000641E0ED0D1F80021002AF9D0C1F80001A7
:10323000A9688E4203D010223046FDF773F80120B2
:1032400070BD002070BD00000C00002000E00040B8
:103250000549064801F11002C0E9001210328260EF
:103260000348016001207047540100200C00002039
:1032700004E500400146024810220068FDF752B8FC
:103280000C0000202DE9F0410446102802D30B4821
:10329000FFF754FE094E0A4D761D204600F07EF8D9
:1032A000070008D0AF4202D13046FFF747FE38464C
:1032B00000F03AF8F1E7BDE8F0810000D00003002B
:1032C000ADDEADDE01480068704700003801002027
:1032D00010B50020114A014600EB40039C186170B4
:1032E000A170D154401CC0B21028F5D3DE22CC21ED
:1032F0000B48FDF729F80A4A0020A2F1180100BF87
:1033000000EB001302EB430341F82030401CC0B235
:103310000628F5D303490620086010BD900A002056
:10332000980B00203801002070B5104C064620682C
:10333000062802D30E48FFF701FE3046FDF798FB42
:1033400018B90B48401CFFF7F9FD0A4D20680A49DF
:1033500055F82000884203D00548801CFFF7EEFD99
:10336000216845F82160491C216070BD38010020AA
:1033700080000300800B0020ADDEADDE10B50446FA
:10338000102802D30348FFF7D9FD034904EB44009A
:10339000085C10BDC2000300900A002070B5002632
:1033A0000446102802D30C48FFF7C8FD0B4D04EB70
:1033B0004404285D70B105F1300000EB8401601910
:1033C00010F8022F51F822600321FFF735FA285D2B
:1033D000401E2855304670BDA2000300900A002010
:1033E00070B50C460646102902D31248FFF7A6FD19
:1033F0003046FDF73DFB18B90E48401CFFF79EFD17
:103400000D4D04EB4404285D032810D205F1300073
:1034100000EB8401601910F8012F41F822600321AC
:10342000FFF70AFA285D401C2855012070BD0020D6
:1034300070BD00008C000300900A002010B5044607
:10344000102802D30948FFF779FD094904EB44002D
:103450000A5C42B101F1300202EB8002084480783C
:1034600052F8200010BD002010BD0000B300030082
:10347000900A00200B4810B50168002479B10A4A6F
:103480000A4B02EB8102491E52F8044D13600160A1
:103490002046FDF7EDFA10B90548FFF74FFD20462D
:1034A00010BD000038010020800B0020ADDEADDE35
:1034B0007800030000487047408100402DE9F74F35
:1034C000904607004FF0000502D13448FFF736FD63
:1034D000334C4FF4803BC4F808B3324EB07818B187
:1034E0002E48801DFFF72AFD706818B12B4809305F
:1034F000FFF724FDDFF8B0A077605FEA08004FF027
:1035000000094FF00108AAF1040724D001282FD0A8
:10351000022829D021481D30FFF710FD86F80280CF
:10352000C4F840910199294489B239603F68C4F8D0
:103530004480DAF80060D4F8400118B117482B3005
:10354000FFF7FCFCAF4215D3AE4201D3BE4221D3FC
:10355000124833301CE0C4F84480DAF80050C4F854
:103560004080C4F84091D9E70F48001D0568D5E7B1
:103570003D68D3E7BE4201D2012000E00020B54201
:1035800001D8012100E00021884203D103483E30E8
:10359000FFF7D4FCC4F804B3BDE8FE8F8600040036
:1035A0000080004010010020448500400048704722
:1035B0004880004070B5144C01266660E660666481
:1035C00012480025056011483C30006810B11048D1
:1035D000FFF7B4FC4FF0FF30C4F80803C4F84051C3
:1035E0000A490420083108600A48456006704570A1
:1035F00085700820FCF7C6FF4FF0E0214FF4807083
:10360000C1F8000170BD0000008000400885004046
:1036100047000400100100200148007870470000B6
:1036200010010020034901200860034900200870B0
:1036300070470000008000401001002070B507486E
:1036400001250561C560064C00260820666066708D
:10365000FCF798FFA670257070BD00000080004048
:103660001001002001484078704700001001002040
:103670000FB408B50399002904D004AA00926A4641
:1036800000F00FF801B05DF814FB10B58268044635
:10369000002A05D0D4E90403216898470020A060DF
:1036A00010BD2DE9FC4791460C00804676D014F8F9
:1036B000011B39B125290ED04046FDF7CFFB2078FC
:1036C0000028F4D198F80C00002867D04046BDE8E7
:1036D000FC47FFF7DABF0020012221782B291BD0FD
:1036E0002D2902D0302908D102E040F0010001E08C
:1036F00040F00200641C002AEFD100252A290ED0D8
:103700002178A1F130020A2A11D205EB850201EBE2
:103710004205641C303DF1E740F00400EAE7D9F8C7
:1037200000100B1DC9F800300968641C0D44217895
:1037300000232E290BD114F8011FA1F130020A2A0F
:1037400005D203EB830201EB4203303BF3E76C2924
:103750000DD068290BD0692921D00BDC252918D080
:10376000582931D063290ED0642915D117E014F8F7
:10377000011FECE7702969D0732932D075291BD05D
:10378000782909D120E0D9F80000011DC9F80010FE
:1037900001784046FDF762FB641C90E76CE0D9F8C5
:1037A00000100A1DC9F800200968CDE900500A225E
:1037B0004046FFF74BF8EFE7D9F800100A1DC9F8AB
:1037C000002009680A2206E0D9F800100A1DC9F88D
:1037D000002009681022CDE90050404603F03AFD70
:1037E000DAE7D9F8001000270A1DC9F800200E6892
:1037F000C00705D112E04046761C7F1CFDF72EFB6A
:1038000031780029F7D104E0202140466D1EFDF7F4
:1038100025FBBD42C0D9002DF6D1BDE74EB13046E3
:10382000FCF7A4FD074604E0202140466D1EFDF78D
:1038300015FBBD4206D9002DF6D103E04046761CAB
:10384000FDF70CFB31780029F8D1A5E7D9F8000085
:10385000011DC9F80010056830214046FDF7FEFA49
:1038600078214046FDF7FAFA08200021CDE9000151
:10387000034610222946B0E7BDE8FC8770B541EA4F
:103880004201DDE904564FF0A04441EA830141EAD8
:10389000052104EB800041EA0641C0F8001770BD25
:1038A00070B541EA4201DDE904564FF0A04441EA17
:1038B000830141EA052104EB800041EA0641C0F89A
:1038C000001770BD70B541EA4201DDE904564FF0C2
:1038D000A04441EA830141EA052104EB800041EA6A
:1038E0000641C0F8001770BD1CB5002100910B46C1
:1038F00001220191FFF7D4FF1CBD1CB500210091EE
:103900000B4601220191FFF7DDFF1CBD1CB5002213
:103910000B46009211460192FFF7C2FF1CBD1CB579
:1039200000220B46009211460192FFF7CBFF1CBD0F
:103930001CB5002100910B46012201911146FFF7B1
:10394000AFFF1CBD1CB5002100910B460122019167
:103950001146FFF7B7FF1CBD4FF0A04202EB8000FD
:10396000D0F8002722F44032C0F80027D0F8002712
:1039700042EA0141C0F80017704701224FF0A0430E
:10398000824011B1C3F808257047C3F80C25704771
:1039900018B5084B6C4601441B68009306E000BF55
:1039A00054F82030D3F81035401C08C28142F7D8B3
:1039B00018BD000010730000034908B50844002139
:1039C00001600068009008BD006000400249405856
:1039D000012800D000207047006000402DE9F04130
:1039E000204D164688460746082801D3042035E0B6
:1039F000B8F1000F03D0202E03D906202EE00320BB
:103A00002CE0384601F06EFA032801D3092025E0A6
:103A1000384600F0FBFF032801D30A201EE000F027
:103A20001BFD022801D2082018E000F0A5FE044684
:103A300006704078324640F0010060704146A01C9C
:103A4000FCF770FCF8B2214601F04EFA10B10120EB
:103A5000BDE8F0810448FFF771FA0F2028700020BC
:103A6000F6E70000CC000020FC0005000149002022
:103A7000486070479C0800200348C1600261012132
:103A80004170002181707047B20000200348C1607E
:103A9000026101214170817070470000B200002076
:103AA00010B500F09DFD18B1BDE8104000F004B85D
:103AB000BDE8104000F092BC7047000010B50B4C00
:103AC000606928B100F042FB0004000C02D005E060
:103AD000022008E0002000F059FE18B100F092FC2E
:103AE000012010BD11202070002010BDCC0000204E
:103AF0002DE9F04116460F46044600F087FF154DAC
:103B000048B157B1204600F08DFF007831688142FE
:103B100005D206201AE00B2018E0032016E020460C
:103B200000F076FF04000DD0A01C0BD02278A11C61
:103B300038463260FCF7F6FB204600F013FE012009
:103B4000BDE8F0810448FFF7F9F90F202870002044
:103B5000F6E70000CC0000202601050010B508287B
:103B600004D3054904200870002010BDC0B200F045
:103B700043FF012010BD0000CC000020084910B513
:103B80004A69527D0AB10C2002E0082803D30420C0
:103B90000870002010BDC0B201F08CF9012010BDEA
:103BA000CC0000200148006970470000CC000020D4
:103BB0000148007870470000CC00002000F01ABDDA
:103BC000082804D3034904200870401F704700F000
:103BD0001DBF0000CC00002001F092B801484068F1
:103BE000704700009C08002001F0A2B810B5012425
:103BF00001F094F9F02815D005DCB0B1042809D003
:103C0000EC2812D110E0F4280AD0F82806D0FC28BD
:103C10000BD101E0002408E0022406E0032404E0C4
:103C2000042402E0052400E00624204610BD70476D
:103C30002DE9F0411D4D064600241D482C70AC6155
:103C40000460446084601B4800F028FC686140B355
:103C5000042000F099FA05F11C00296900F068F8C9
:103C60000746304600F0B8F800EA0706002000F0EA
:103C700099F80640012000F0E5F80640022000F027
:103C800079F80640002000F0FFF80640012000F01F
:103C9000A1FE0020EC6000F05FFD16B10120BDE840
:103CA000F081012028700020F9E70000CC000020FE
:103CB0009C080020A92D000001484069407D704704
:103CC000CC00002070470000084A10B553695B7DA6
:103CD0000BB1022002E0082803D30420107000205A
:103CE00010BD00F063FD012010BD0000CC000020DD
:103CF000064910B54A69527D1AB1022008700020A9
:103D000010BD00F029FA012010BD0000CC000020F9
:103D1000064910B54A69527D1AB102200870002088
:103D200010BD00F025FA012010BD0000CC000020DD
:103D300010B50F4C6269527D0AB1022014E01029BF
:103D40000FD871B178B10A462161014608481C308C
:103D5000FCF7E8FA064821691C3000F029FA012036
:103D600010BD072000E003202070002010BD0000DF
:103D7000CC0000200A4910B54B69024601205B7D4A
:103D80000BB1022004E0012A05D0022A04D00E2043
:103D90000870002010BD002000F088FA012010BD3E
:103DA000CC0000200A4910B54B69024600205B7D1B
:103DB0000BB1022003E032B1012A03D00E200870BB
:103DC000002010BD012000F0EDF9012010BD000021
:103DD000CC00002000F014BC10B540B1012808D080
:103DE00002280BD0064905200870002010BD0120D4
:103DF00000E0022000F00AFC012010BD0020F9E7DD
:103E0000CC000020064910B54A69527D1AB1022043
:103E10000870002010BD00F079FF012010BD0000E7
:103E2000CC000020064910B54A69527D1AB1022023
:103E30000870002010BD00F081FF012010BD0000BF
:103E4000CC000020014610B50020072914D2DFE87D
:103E500001F0040F06080A0C0E00042008E0FC2004
:103E600006E0F82004E0F42002E0F02000E0EC207E
:103E700001F05AF8012010BD02490E200870002000
:103E800010BD0000CC0000200A4910B54B69024665
:103E900000205B7D0BB1022003E032B1012A03D088
:103EA0000E200870002010BD012001F047F801200D
:103EB00010BD0000CC00002010B5FFF7FDFE00286B
:103EC00006D0FFF7EDFD30BFFFF7F6FE0028FBD16F
:103ED00010BD000038B50446012181F3108820256B
:103EE00005E06A46064920460095FFF701FE204698
:103EF000FFF766FE0028F4DC002080F3108838BD50
:103F0000600800200149002048707047B20000207E
:103F10000149002088707047B200002001484078B5
:103F200070470000B2000020014880787047000010
:103F3000B200002010B501F0F3F903490020086138
:103F40000249087010BD0000F4080020F8000020AD
:103F50002DE9FE434D4800684D4C012802D04D48E4
:103F6000006828B960680078202801D8012100E0A5
:103F70000021494E03204FF0000830704348C4F838
:103F8000008008300568424F183F89B300684149F6
:103F90000839086002A8CDE900043C480C300268EA
:103FA00001232946184602F067F910B3012805D00D
:103FB000022821D0032855D0384851E0029818B182
:103FC00036481C38FEF7BAFF284602F0B8FA18B98E
:103FD00032481B38FEF7B2FF01F0D6F9B97D002355
:103FE000CDE900017068EAB290F9161018461CE09D
:103FF0001EE02A48113833E0029818B927480D38D6
:10400000FEF79CFF284602F09AFA18B923480C38AC
:10401000FEF794FF01F0B8F9B97DEAB2CDE90001ED
:104020007068012390F91610029800F07DFB19E0EA
:1040300000F072FE30B101F0A7F90146BA7DE8B296
:1040400000F044FB0023CDF800801A4619461846BC
:10405000CDF8048002F010F9042803D00F480F3087
:10406000FEF76CFF206838B1012060750C482061B4
:1040700004203070BDE8FE8301F052F984F8158009
:10408000C4F8108000F00EF8F4E7000000140040BF
:10409000F408002034150040F80000204406090010
:1040A0003D41000070B5FFF745FF1F4D012028700E
:1040B0001E4801681E4A21F0FF0112691143016088
:1040C00002F046FA1A4C4C3410B302F041FA0328BD
:1040D00002D01848FEF732FF022001F05FFB0020FB
:1040E00001F0B4FB02F034FA032803D01148083081
:1040F000FEF724FF2878012803D00E480E30FEF783
:104100001DFF02202870002020610B48E06070BD78
:1041100002F012F80228DFD302F040F960600028B4
:10412000DAD10448401FD5E7F800002030150040E0
:10413000A8080020F4050900513F000002490520AD
:104140000870FFF7AFBF0000F80000200148006AC8
:1041500070470000A8080020034910B5086200F06D
:10416000ADFD0249086010BDA80800201C150040E4
:10417000034910B5486200F0A1FD0249086010BD76
:10418000A8080020201500400449487704490A681F
:1041900022F4E02242EA004008607047A8080020AC
:1041A000181500400149087670470000A808002053
:1041B00070B50C00054602D10748FEF7BFFE1DB9D9
:1041C0000548401CFEF7BAFE0448C0E90145BDE8B9
:1041D00070400020FEF74EBFB30309000C09002019
:1041E00010B500F099FD044901F1640208B1C868F6
:1041F00000E08868106010BDA80800201CB51049B8
:104200004FF44070086002F0A3F9012812D0022890
:1042100010D0032813D10020009003460246014627
:10422000019002F029F8042809D0BDE81C40054897
:10423000FEF784BE0021084602F0CEF8F3E71CBD6D
:1042400008F5014048020900144981F83100144979
:104250000A6822F0FF020A6048B1114A0B1D0832B9
:10426000012807D002280ED00E48FEF767BE086866
:1042700008607047086840F001000860FF20106087
:1042800040F2071007E0086840F0020008604FF6AF
:10429000FF7010600448186070470000A8080020F4
:1042A000341500402E04090021100100044981F852
:1042B0003200044908B1012800D1086070470000AD
:1042C000A8080020101500402DE9FF413E48006875
:1042D000012802D03D48006830B93D484068007868
:1042E000202801D8012700E0002700F0F5FB384C1A
:1042F0000126183C00B9266102F02AF9012802D0F3
:104300003448FEF71BFE344D6868007D18B1314813
:10431000401CFEF713FE01F003F8EFB3012108463D
:1043200002F05AF820B1012828D0022826D10FE047
:1043300001F02AF8064601F067FFC7B201F05EFF00
:104340008446A07D0021CDE90260CDE900710DE039
:1043500001F01AF8804601F057FFC7B201F04EFF96
:10436000A17DCDE90076CDE9028184466868628945
:10437000218990F91630604600F0B8F9FEF774FE16
:10438000E06013484C3840696060FFF729FF04B0D3
:104390000020BDE8F04100E001E0FEF783BE6E7052
:1043A00000F0BAFC00280CD000F0EEFF054601F04A
:1043B0002BFFA27D04B02946BDE8F041C0B200F059
:1043C00085B9BDE8FF8100000014004034150040AD
:1043D000F408002037070900F800002010B501207C
:1043E00080F310880648417D29B1817819B90121EF
:1043F000817000F03FFB002080F3108810BD0000AA
:10440000DC08002070B5124C607D00281ED100F041
:10441000C3FA04F13005A86810B90E48FEF78EFD06
:10442000686818B90B48401CFEF788FD02F0C0F818
:1044300018B10848801DFEF781FD002002F0D8F871
:1044400001206075BDE8704000F014BB70BD000035
:10445000DC080020CE02090001F0E2BE30B50D4DAF
:1044600085B0687D002813D000F042FB00F058FFB3
:104470000024AC706C7505208DF80000684601F0D2
:1044800007FE0548047005B0BDE83040FFF7B6BE32
:1044900005B030BDDC080020F80000202DE9F04117
:1044A0000546012080F31088484E4FF00308002491
:1044B000707086F80080B470746034817481F46028
:1044C00007463461347506F1180074750460446061
:1044D0008460C46004610475183084604460FFF730
:1044E00069F8284601F00EFE01F09CFE002002F063
:1044F00071F806F13000FEF7E7FD00210820FCF717
:1045000083F800210120FCF77FF801211520FCF73A
:104510007BF8012000F07AF8A6F13405FF2028612D
:10452000042068772A4929622A49696285F8287037
:10453000022185F8291085F82A8085F82B000520AE
:1045400085F82C00062085F82D00072085F82E0020
:10455000082085F82F0085F8304085F8311085F85F
:104560003270692045F8140B1E2028604FF4167035
:1045700045F8100C022000F091FC0F2000F094FC94
:10458000EC802F716F712C72204601F043FE707821
:10459000012802D01048FEF7D1FC3770B470746067
:1045A00034817481F46034610C48347574758460AE
:1045B000447000F0F1F90820FBF7D9FF1520FBF754
:1045C000D6FF84F310880148BDE8F081DC080020A4
:1045D00004070A0D05080B0E9F020900F8000020D1
:1045E0000348407D08B1002070470120704700005B
:1045F000DC0800200148408B70470000A80800201C
:104600000149488370470000A808002010B5012127
:1046100081F3108807490A78824204D04870487DA7
:1046200028B100F027FA002080F3108810BD00F0B8
:1046300003F8F8E7DC08002030B5224D85B0287873
:10464000697888423BD008B900F0A6F9687808B9C3
:10465000FFF7D4FD1C480024046000F061FE1948F7
:1046600018300460446004618460C46028780128C4
:1046700002D0022808D015E001F06AFF90B10021B5
:10468000084601F0A9FE0DE0FFF754FC01F060FFC1
:10469000032807D1002300941A46194618460194AE
:1046A00001F0EAFDFFF79CFD6878287004208DF882
:1046B0000000684601F0ECFC012005B030BD002090
:1046C000FBE70000DC08002054F5014000B585B090
:1046D00006238DF806208DF805108DF804008DF85E
:1046E0000030684601F0D4FC05B000BDF0B585B0DF
:1046F0000DF1280C9CE8F0008DF80C308DF80D4081
:104700004FF0000C0190ADF808108DF80E508DF8A8
:1047100000C0ADF80A208DF80F608DF81070684663
:1047200001F0B6FC05B0F0BD70B586B00226DDE93B
:104730000A458DF808108DF8092001908DF80A308F
:104740008DF800608DF80C508DF80B40684601F034
:104750009FFC06B070BD00000149886070470000F2
:10476000F800002010B5012181F3108801F080FDD0
:10477000002080F3108810BD10B5012080F3108850
:1047800001F078FD002181F3108810BD10B50446BA
:10479000082802D30348FEF7D1FB0348204490F8D1
:1047A000280010BDAD030900A808002070B5082836
:1047B00019D20F4A024482F828108207D40EFF2231
:1047C000A240D243042801D20A4D01E0094D2D1D1B
:1047D000286810402860084600F05EFA2968A0406A
:1047E0000843286070BDBDE870400348FEF7A6BBD3
:1047F000A808002024150040A703090010B51B4C91
:1048000000206070FEF71CFC19490860FEF72CFCC4
:104810001849887501F09CFE012807D001F098FE28
:10482000022802D01448FEF789FB002000F0B6FFF2
:10483000FEF740FE114908606068091D4068086085
:10484000A068002811D0007820B1FEF733FEA168DF
:1048500000F002FCA0680179002906D000F0D0FB2E
:10486000A068BDE8104000F0D9BB10BDF8000020E2
:1048700008150040DC0800209706090050F50140AB
:1048800010B501F00FFE002820D011480021018151
:10489000418101F0B9FC0F49086001F0B5FC01212C
:1048A00081400C48001D026822F0FF0211430160A4
:1048B00001F0A4FC064C1834206001F099FC606003
:1048C0000548E060BDE81040FFF798BF10BD00004C
:1048D000DC0800202C150040C942000015480021CA
:1048E0000160012101601448016821F480710160B8
:1048F000016821F00F01891D0160016821F4702118
:1049000041F440310160001D016821F00071016037
:10491000016841F080710160016821F0FF0141F000
:1049200020010160016821F47F4101600120FBF753
:104930001EBE0000FC1F00401415004070B5134C53
:104940001348A16800F096FE6060114C4C3C607FFB
:10495000FFF71AFC206AFFF7FFFB606AFFF708FC0D
:104960000025601990F828102846FFF71FFF6D1CDE
:10497000082DF6D3074914F8300F08606078FFF768
:1049800063FCA078BDE87040FFF790BCF800002001
:10499000F40800200C1500400C4910B500200860F8
:1049A0000A484FF440744C380460FFF797FFFEF755
:1049B000FDFD064908310860091F054808600348E5
:1049C00050380460BDE81040FFF7B8BF54F501400F
:1049D0000411004010B504460448406810B904486A
:1049E000FEF7ACFA0348047510BD0000F800002083
:1049F0006E040900F408002010B5012181F310882D
:104A000001F09AFD002080F3108810BD01F097BDE1
:104A100010B5012181F3108801F094FD002181F38C
:104A2000108810BD01F091BD0349012208610146C3
:104A30000248FEF743BD0000DC080020BD65000011
:104A400070B50C4601F0D4FD074D2869A04202D391
:104A50000648FEF773FA28690122211A0448FEF776
:104A60002DFD0020286170BDDC080020D60609005D
:104A7000BD65000010B5FEF7CFFD012822D101F081
:104A8000B1FD10B11048FEF759FA002264210F4819
:104A9000FEF714FD0E48007F80B90E480121016029
:104AA00000220007C0F80021016000BF00BF00BF66
:104AB000AFF30080D0F800110029FBD0BDE8104012
:104AC000FEF7B0BD10BD0000B4060900BD650000D2
:104AD000A808002014050040044810B5006918B962
:104AE000FEF7C0FD002800D0012010BDDC0800202A
:104AF00010B5FEF791FD01280ED0FEF79FFD074887
:104B0000007F10B9012081074860002001F070FD8E
:104B1000024900203431486010BD0000A808002080
:104B20000B4810B54068407D30B1012000F08EFE8A
:104B300008490889401C0881074900200860054889
:104B4000343803C8BDE81040091A0020FFF778BFC9
:104B5000F8000020DC08002054F5014070B586B054
:104B6000FFF7BAFF494D4A4E05F1340458B100F041
:104B7000BDF8A078002869D0FEF7B8FA06B0BDE805
:104B80007040FFF76BBC2078012802D0022804D0C7
:104B900008E000F017FF28B170E0307804286DD0ED
:104BA00003286BD0FEF7A2FA00F0A0F8A07868B155
:104BB000FFF754FC01F0C0FA022840D303208DF81F
:104BC0000000684601F064FA06B070BDFFF734FDDE
:104BD00020B100206968FFF733FFEBE72078F0B1E0
:104BE000012816D0022817D02A48FEF7A7F9687EB8
:104BF0000128DFD100F090F80028DBD12078D8B16F
:104C0000012811D00228D5D022481A30FEF796F993
:104C1000D0E700F099F8EAE700F01AF9E7E700209A
:104C20006968FFF70DFFE2E701F092FC0028C1D1AF
:104C300001F00CFC0028BDD1FFF75AFFBAE706B01F
:104C40001448BDE870403630FEF778B92078022865
:104C500008D0FEF74BFA696806B00020BDE8704046
:104C6000FFF7EEBE3078042808D0032806D0FEF700
:104C70003DFA06B0BDE8704000F0EAB8686806B0DA
:104C80004008BDE87040FFF7CFBE0000A808002034
:104C9000F8000020D0040900024610B500200146AB
:104CA00022FA01F303F00103C1F10704A340034317
:104CB000491CC9B2D8B20829F2D310BD2DE9F04180
:104CC0000024064625461827E80026FA00F0C0B260
:104CD000FFF7E2FF694207EBC101884020436D1CEA
:104CE000EDB20446042DEFD3BDE8F08103484168DE
:104CF00009B1491E4160FFF773BA0000DC080020CB
:104D00000148406970470000A80800200149486137
:104D100070470000A808002004480178022902D04A
:104D20004068002800D0012070470000DC08002007
:104D30000148406870470000A80800200149486009
:104D400070470000A80800202DE9F04186B000F06F
:104D5000E7FA01F0FDFB3A4D05F1340420B3688B0E
:104D6000B0B3218981423BD30121002001F034FB03
:104D700001F044FA26898046648901F045FA074625
:104D800000F002FB014601208DF80000ADF808603C
:104D90008DF80C70CDF80480ADF80A408DF80D1038
:104DA000684601F075F944E001F0C6F9022840D3E5
:104DB000FFF7B2FF68B1FEF76FF9D0BB287E20B9CC
:104DC000FEF752F9E168884233D1FFF759FD30E030
:104DD00006E0E068FEF74EF90020FEF763F9F4E71D
:104DE000FEF740FC10B11748FEF7A8F8FEF728F9C7
:104DF00015490968884202D06089401C60811348C7
:104E00004078A0B9FFF788FF88B101F0FDF90646A8
:104E100000F0BAFAA17D8DF806108DF80500072282
:104E20008DF800208DF80460684601F031F9FFF735
:104E3000E5FC296806B00120BDE8F041FFF700BE9F
:104E4000A80800207C05090008150040F800002093
:104E500070B50024FEF7F4F80D4D2968884207D09C
:104E6000FEF7EEF82860FEF7FFF80A49012488757E
:104E70000948641E0078044201D1FFF713F9054880
:104E800034384168BDE870400020FFF7D9BD00000C
:104E900008150040DC080020F80000200149C86027
:104EA000FFF79EB9A808002001498860FFF798B96C
:104EB000A808002010B50446012181F31088074896
:104EC000017821B1407D10B10548FEF737F8204642
:104ED00001F044FB002080F3108810BDDC080020A6
:104EE0006803090001F043BB10B5012282F310886A
:104EF00001F04AFB58B10848817819B9407D08B1E2
:104F0000FFF7B8FD002080F31088012010BD0020BD
:104F100080F3108810BD0000DC080020014890F8E4
:104F200030007047A8080020024981F8300002498B
:104F300008607047A80800200C1500400149087758
:104F400070470000A808002070B51149114A0025DB
:104F5000487802EB0010027B22B10F4AD2F80C21F4
:104F600002B10125807A0870012000F0DFFB0B4CB4
:104F70001DB1A068806800B180476068002806D035
:104F80000179002903D0BDE8704000F01BB870BD66
:104F9000180900208873000000100040180100204C
:104FA00007480069012805D0022805D0032805D14B
:104FB00000F09AB800F04CB900F0E4B87047000077
:104FC00018090020827B002193000B4A1344C3F888
:104FD0001019C37B02EB8302C2F81019427B012136
:104FE000837BC07B01FA02F201FA03F3814003489C
:104FF0001A430A430260704700F0014008F501407F
:105000004279054BC079012103EB80000AB10166AA
:105010007047016370470000006000408268002113
:10502000C2F84011C17B094ACB0009490B44C3F8BF
:105030001025C37B826801EBC301C1F81425C17B35
:1050400001208840034908607047000010110040AB
:1050500000F0014004F501402DE9F0410746886861
:1050600000260C46C0F840618868097B1A4D00F59F
:10507000A07005EBC101C1F810056278E178207BD2
:1050800000F08EFC607B05EBC000C0F81075617B02
:10509000A06805EBC101C1F814051048C0F80C6107
:1050A000C0F81061A17B0E4805EBC101C1F81005E5
:1050B0006278E178A07B00F061FC217B0120627BBB
:1050C00000FA01F100FA02F21143A27B9040014381
:1050D00004480160BDE8F08100F00140001000408C
:1050E0000C11004004F501402DE9F0411F4E022053
:1050F000002530700320707075603575B0691C4CE8
:10510000401CB061C4F80C51C4F80051C4F81051EF
:10511000C4F80451C4F82851C4F80052681EC4F8F9
:1051200008030120FBF739FA124FB868007D50B12F
:10513000114800684042B075C4F81C510120A061BC
:105140000E49800208600C4844380068F1688842C3
:1051500002D00B48FDF7F2FEB868C068002802D004
:10516000BDE8F0410047BDE8F081000018090020CB
:1051700000100040180100204815004008F50140CB
:1051800051040A0010B52D4CD4F80C01012802D0AE
:105190002B48FDF7D3FED4F81001012803D028488E
:1051A000401CFDF7CBFED4F80001012803D02448B1
:1051B000801CFDF7C3FED4F8040118B12048C01CC0
:1051C000FDF7BCFE0020C4F80C01C4F81001C4F8BF
:1051D0000001C4F80401C4F808010221C4F8001257
:1051E0000121C4F808130822C4F80423154A032334
:1051F000154C137010755060606890B1027912B14F
:10520000FFF7E0FE0DE002785AB1027B437B807B22
:1052100001FA02F201FA03F381400C481A430A43EF
:105220000260A068006900B18047A068806800281B
:1052300002D0BDE81040004710BD00000010004043
:10524000F3030A00180900201801002008F50140A6
:105250002DE9F0412A4DD5F80001012802D0294856
:10526000FDF76CFED5F80401012803D02548401C49
:10527000FDF764FE24480168244801700021C5F848
:105280000011C5F80411C5F80811491EC5F8081326
:105290000126C5F8046381681D4F097D09B1B1027B
:1052A0003960446814B3207900B3617BDFF864800F
:1052B000A06808EBC10100F5A070C1F81005627983
:1052C000E179607B00F06CFB607B06FA00F03860EF
:1052D000207B114908EBC000C0F810156279E17914
:1052E000207B00F04BFB207B86403E600B4806494C
:1052F000091FC06808600B20C5F80002BDE8F081F6
:1053000000100040BD030A000815004018010020ED
:1053100004F5014000F001400C1100401809002084
:1053200070B50120FBF744F90120FBF736F9144C66
:105330004FF0FF30C4F808030026C4F80062C4F838
:10534000106101202061A0610E4D2878012813D042
:10535000022813D0032811D05FF00100FDF7DCFE16
:10536000C4F810612E706E75002000F0DFF9BDE802
:1053700070400120FBF732B90620EFE70220EDE78D
:105380000010004018090020014800787047000014
:105390001801002001F01F014FF4003343EA0121FE
:1053A000830009481844C0F81015D0F810150AB940
:1053B00041F48011C0F81015D0F8101541F0030128
:1053C000C0F81015704700000060004008480069F0
:1053D000012806D0022806D0032806D00548FDF78C
:1053E000ADBD00F095B800F007B800F0F1B80000CE
:1053F0001809002033050A002DE9F047DFF8F08096
:105400000421012088F80010D8F81810491CC8F8A9
:105410001810FBF7C2F837480068374D2870374C32
:105420000026C4F80C61C4F80061C4F81061C4F827
:105430000461A868DFF8C8900127007DA0B130485A
:1054400008380068400502D42E48FDF777FD29484A
:1054500040300068404288F81600C4F81C61A7611B
:105460004FF48061C9F80010D4F8000118B1254844
:105470000930FDF763FDD4F80C0118B121480A305A
:10548000FDF75CFD4FF0E020B046D0F8000210F0D0
:10549000020F03D01B480B30FDF750FD6E68CEB1F4
:1054A0003078B8B1C4F80C81717B184A164802EB09
:1054B000C101C1F810057278F178707B00F05EFAD6
:1054C000707B0F4907FA00F0091F0860F07B8740E6
:1054D000C9F80070A868C06800B18047A868417D1D
:1054E000002903D003490068091F0860BDE8F08760
:1054F0001809002008150040180100200010004085
:1055000008F50140C0040A000C11004000F0014001
:105510002DE9F041294C0026C4F80C61C4F8006163
:10552000C4F81061C4F80861C4F80461012004F5EE
:105530008074FBF732F80820C4F804020125C4F88F
:1055400008520720C4F800011D484468002C32D0DE
:10555000207920B1207B1B4905FA00F008602078F3
:10556000002828D0A068C0F84061A17B164FA06831
:1055700007EBC10100F5A070C1F810056278E17871
:10558000A07B00F00DFAA068C0F84061E17B0F48F5
:1055900007EBC101C1F81005E17BA06807EBC10171
:1055A000C1F81405A17B05FA01F0E17B8D400549A6
:1055B0002843091F0860BDE8F0810000001000408A
:1055C0001801002008F5014000F001400C110040D6
:1055D00070B5234CD4F80C01012802D02148FDF706
:1055E000ADFCD4F81001012803D01E48401CFDF783
:1055F000A5FCD4F80001012803D01A48801CFDF74F
:105600009DFC0020C4F80C01C4F81001C4F800018E
:10561000C4F80401411EC4F80813C4F80002124C77
:10562000626872B1117861B1557B012303FA05F10B
:10563000957BD27B03FA05F593400C4A2943194325
:1056400011600B49032208704A7048600875A06811
:105650000069002802D0BDE87040004770BD00001E
:1056600000100040F5040A001801002008F5014070
:105670001809002070B506460C460120FAF798FF7D
:10568000FFF74EFE244D25482649C5E90146002472
:105690000470032646704460046104754475847583
:1056A0001F4808601E48F030091F08601E48016846
:1056B00021F0010141F0807101600120FAF78EFFB5
:1056C000686838B3017909B9017819B38168C1F8FC
:1056D00008650422C1F81025027CC2F18102C1F8DC
:1056E000402540F20112C1F80022C1F80445012210
:1056F000CA60C1F84041017921B142798179C0790C
:10570000FFF748FE6868017821B142788178C07857
:10571000FFF740FE014870BD180100201809002065
:105720001410004064F50140741700402DE9F04169
:10573000174C00250746C4F80052164E307803284F
:105740001CD0681EC4F80803C4F80C510320707004
:105750000120FAF722FF00BFC4F80051C4F810512D
:10576000C4F8045175603575002F0FD00A48806861
:10577000006900280AD0BDE8F04100476FF008003A
:10578000C4F808030820C4F80403E5E7BDE8F08185
:105790000010004018090020180100202DE9F047F2
:1057A0000746DFF8908022484FF0FF3100EB0716E4
:1057B000C8F808130120FAF7F0FE1F4C0025DFF8A7
:1057C0007C9065756770D9F80800032F0268A260A5
:1057D0004168C4E90315A5613068606019D2337A65
:1057E000C8F80032C8F80C51C8F81051F37A1448C0
:1057F0001BB10160006828B108E00260006828B9A8
:10580000104801E00F48401DFDF798FB717AC8F879
:105810000413D9F80800007D28B1022F03D10A49EA
:10582000A5757802086001206075BDE8F08700006A
:1058300088730000001000401809002018010020A3
:10584000041500409C020A0004F501402DE9F05FB8
:10585000404C82464048667800EB0617607D012880
:1058600002D03E48FDF76AFB207D18B13B48401C42
:10587000FDF764FB012500212575DFF8E490A046C3
:105880006175032E47D2BAF1000F3CD1D9F804401C
:10589000BCB32279AAB38A460846A168C1F8400180
:1058A000217BDFF8C0B0A0680BEBC10100F5A07050
:1058B000C1F810056279E179207B00F071F82A497E
:1058C000C1F80CA1607B29490BEBC000C0F8101592
:1058D0006279E179607B00F051F8217B627B05FA07
:1058E00001F005FA02F1084321490860D9F80400E3
:1058F000204A81791268CA4012F0010F01D18068F4
:10590000056038680560022E01D0012E07D1B97AF2
:1059100088F8001003E011482530FDF70FFBD9F897
:105920000800007D002813D0022E11D11048006815
:10593000400503D409482A30FDF700FB0E480068F3
:10594000002805D1BDE8F05F04482B30FDF7F6BA1A
:10595000BDE8F09F1809002088730000B8020A0013
:105960001801002000F00140001000400C11004020
:1059700004F501401005005004150040064B03EBF0
:10598000C0000AB1054A01E0044A303A02EB810145
:10599000C0F814157047000000F00140606000403E
:1059A000064B03EBC0000AB1054A01E0044A30325D
:1059B00002EB8101C0F814157047000000F00140AF
:1059C000306000400348D0F80401012800D00020D6
:1059D000704700000010004030B5124B0146002017
:1059E000D3F81044224609E0157A854205D1401CBF
:1059F0000A28F7DB4FF0FF3030BD5268002AF3D1A0
:105A0000421CF9D00872D3F810242AB152684A60B7
:105A1000D3F81024516030BD0022C3F810144A603E
:105A200030BD00003C040020F0B595B01C46154682
:105A30000F4608461A9E00F009FB182109A8FAF73C
:105A40008AFC0E96CDE909540023082203A93846A2
:105A500000F011FB05980690BDF81000ADF81C0091
:105A6000BDF81200ADF81E0000208DF8210003984B
:105A7000082600F00300012802D0022818D032E0E6
:105A800003983346850AC0F3C2008DF820000398BE
:105A90000FA9C0F38314A200384600F0ECFA09A85D
:105AA000009006AB22460FA9284600F02BFA1AE018
:105AB0000398840DC0F3C2008DF82000082C01D299
:105AC000254600E0082533462A460FA9384600F04F
:105AD000D2FA2E44641B09AB06AA29460FA800F08F
:105AE00063F9002CEAD1384600F0B6FA15B0F0BDE3
:105AF0007047012001F060BA084810B50178084AE3
:105B0000515C19B1001D00F091FF02E00C3000F073
:105B10009FFEBDE81040002001F04EBA3C0000207E
:105B20000000002008B5034A00924023024AFFF714
:105B30007BFF08BDE56C00003C0300200A4A0129F8
:105B400002EBC00007D0022907D0032907D004299F
:105B500007D000207047022070470420704700796A
:105B60007047407970470000FC74000010B5FFF7E3
:105B7000C0FF04210348FFF72FFF024901204872AC
:105B800010BD0000500000202DE9F0478CB0FBF75D
:105B900075F918B100200CB0BDE8F087784C0020F2
:105BA000C4F81804BFF34F8F60680290A5684FF0E7
:105BB0000008284004EB800008E021680298814238
:105BC00001D86160E6E7284004EB80000C3002A9B0
:105BD000FCF7D0FE0028F0D103AB029901EA0502E0
:105BE00004EB8202491CD26843F82020401C029139
:105BF0000228F2D3039800F00300022802D0012803
:105C00004ED0A5E003985022810D8946B2EB905FFB
:105C100000D850210E4666F39F5003900831594832
:105C200000F0CBF9070078D000F010FA43460822C4
:105C300003A9384600F025FA029908F1080A29401C
:105C4000681A8000001D864223D94D4D0C3530B1B5
:105C5000C2B204EB8101301A90460C3104E02946AF
:105C6000F2B2002590462846C6B25346384600F0A8
:105C700008FA0AEB08032DB1324629464FEA07001D
:105C800000F0FFF9029909F1030001EB9000029086
:105C90003AE004EB81015346324638460C31EFE7D7
:105CA0000398C0F38311062900D3062161F38910FC
:105CB0000390C0F38310801C8100324800F07DF90E
:105CC000070045D000F0C2F94346082203A9384630
:105CD00000F0D7F908F1080800260FE002984346C3
:105CE00000EA0501401C04EB8101029004223846C1
:105CF0000C3100F0C6F908F10408761C0398C0F3D3
:105D00008310B042EAD847B1D4F81054D4F818043C
:105D100068B1384600F0A0F92CE019E0687A012853
:105D200004D12A6828463946126890476D68002DCC
:105D3000F4D1384600F090F90020FAF754FFD4F877
:105D4000180408B9029860600020FAF74EFF11E0CD
:105D5000D4F8104404E021682046896888476468C4
:105D6000002CF8D108480221008801EB004007A16F
:105D700000F016F8FBF782F880F001000BE7000056
:105D80003C0400202C750000500100204261636B30
:105D9000656E647320666C7573686564000000004E
:105DA00000231A4600F0BEBF2DE9F0470E4680469C
:105DB0001C46924608293ED894F80C900020207387
:105DC0001946104600F0E8FE0025B54206D218F844
:105DD00005201AA12046FDF74BFC03E019A120463F
:105DE000FDF746FC6D1C082DEFD317A12046FDF7EB
:105DF0003FFC0025B54210D218F80570FAF78EFA6C
:105E00000068C05D10F03E0F01D03A4600E02E223F
:105E10000EA12046FDF72CFC03E00DA12046FDF766
:105E200027FC6D1C082DE5D301222146504600F0C9
:105E300095FE84F80C90BDE8F087000020253032F4
:105E400078000000202020007C0000002563000076
:105E500020000000104810B5FF2181600021016082
:105E60004160C0F81814C0F8141480F820140B48CE
:105E700000F0F0F800280DD109480A490A4B401AF1
:105E8000C108002003E000BF23F82000401C884226
:105E9000FAD3002010BD00003C0400202C75000047
:105EA0002C750000FC7400003C01002002480349EE
:105EB000401AC008704700002C750000FC740000F8
:105EC00013B56846FCF758FF08B100201CBD024816
:105ED000009950F831001CBDFC74000070B50848F2
:105EE0000125D0F8104480F8205405E0657221683F
:105EF0002046496888476468002CF7D170BD0000CF
:105F00003C0400202DE9FF4781460C9D00200C46F3
:105F10002F7B2873984616462946184600F03CFE0B
:105F2000072E42D2DFE806F004090F161F2A3600BA
:105F300049462846FDF79CFB37E04946284622683B
:105F4000FDF796FB31E0D4E9002349462846FDF7EA
:105F50008FFB2AE0A0680090D4E900234946284638
:105F6000FDF786FB21E0D4E90201CDE90001D4E987
:105F7000002349462846FDF77BFB16E004F10800A4
:105F800007C88DE80700D4E9002349462846FDF7F5
:105F90006FFB0AE004F108000FC88DE80F00D4E998
:105FA000002349462846FDF763FB00222946404668
:105FB00000F0D4FD2F73BDE8FF872DE9F041858AFD
:105FC00080462D1F4819C01CB0FBF5F0C6B24046F4
:105FD000FCF7D8FF041E19D0002020710120607149
:105FE000E58000272546761EC4F800800BE0404679
:105FF000FCF7C8FF60B16179491C617128600546F2
:106000007F1CC0F80080B742F1D32046BDE8F08184
:10601000204600F002F80020F8E72DE9F04145792C
:1060200001466B1E002201E00968521C9A42FBD314
:106030000F680146002605E038460C68FCF7C1FFF2
:106040002146761CAE42F7D3BDE8F0810121001D48
:10605000FCF77CBFFCF7CABF10B504460121001D48
:10606000FCF78AFF10F0FF0F04D12046BDE8104076
:10607000FFF7D3BF10BD38B501240094FCF740FEF4
:1060800038BD38B500240094FCF73AFE38BD000056
:1060900070B51A4C0546206810B91948FCF74EFF38
:1060A000D4F8D4000A2803D31548401CFCF746FF57
:1060B000D4F8CC0000EB800004EB800115F8040B51
:1060C00008712DCD8860CA600B614D61D4F8D40091
:1060D000401CC4F8D400D4F8CC00401CC4F8CC0058
:1060E000D4F8CC1000200A2901D3C4F8CC004FF01A
:1060F000E0214FF40010C1F8000270BD3409002007
:106100004A000B0010B5040002D10948FCF716FF45
:10611000084941F8CC4B002041F874098867C867EA
:106120004FF0E0214FF40010C1F8000110BD000055
:106130003E000B003409002010B5074CD4F8D40001
:106140000A2802D90548FCF7F9FED4F8D400C0F1BA
:106150000A00C0B210BD00003409002079000B0015
:10616000094902220A60BFF36F8FBFF34F8F0A1DE8
:10617000106006480268002AFCD000200860BFF3C7
:106180006F8FBFF34F8F704704E5014000E401407B
:1061900010B500F003029043D200FF24944003683E
:1061A0009140A343CA18094901230B60BFF36F8FC5
:1061B000BFF34F8F026006480268002AFCD000201F
:1061C0000860BFF36F8FBFF34F8F10BD04E5014030
:1061D00000E40140F0B515460E460746002404E0F1
:1061E000315D3819FFF7D4FF641CAC42F8D3F0BD21
:1061F0000148C068704700000C0A00200148806810
:10620000704700000C0A00200148406870470000F9
:106210000C0A0020014981F8810070470C0A002017
:10622000FDF750B870B5FDF753F800240E4E254623
:10623000204600F053FC04F1080000F04FFC3555F7
:10624000641C082CF4D30948012105704560856061
:10625000C5600561456180F8805080F85850C56779
:1062600080F8811070BD0000240100200C0A00207D
:10627000FDF75AB8FDF7FEB82DE9FF4F81B0444F46
:10628000DDE90EA803260025F86F0C46AB4610B9D1
:106290004048FCF753FE3878032803D03D48401CA3
:1062A000FCF74CFEF86FB9464178C8072FD199F832
:1062B000810060B300270198E8B3039A584662F35F
:1062C0001700C1F3410161F31F6009EB84018A6B80
:1062D000CAF800B0C8F800B00090904234D0204610
:1062E00000F024FC051E07EA05072DD004F1080183
:1062F00009EB81020099916104990D4223D0264E49
:10630000305D00B3204600F032F910B105E00127FE
:10631000D1E720482830FCF711FE204600F029F98B
:10632000CAF80000BAF1000F0AD018B919482E3087
:10633000FCF704FE00E01BE006F804B0022603E0D0
:1063400014483230F4E7012677B1204600F02DF9E9
:10635000C8F8000018B110480121015506E00C48AA
:106360005830C8F8000001E0C8F800B00DB107E0EF
:1063700004264C46D9F87C00FCF7D6FFC4F87CB064
:1063800089F800B000F068F805B03046BDE8F08F3D
:106390000C0A00202D010C002401002010B50C4C2B
:1063A000207810B10B48FCF7C9FD00F0B3FB0028C2
:1063B0000DD0FF220270417841F0060141700021AA
:1063C0004318491C9A702029FAD30321217010BD6B
:1063D0000C0A002007010C0070B51A4C05460E4649
:1063E0002078012804D0022802D01748FCF7A6FD27
:1063F000B5B12078012803D01348401DFCF79EFD5D
:10640000E06818B91048801DFCF798FDE068007836
:1064100020B1606800F08AFB022502E0002500E060
:1064200004254EB1606800F0A4F8A168814203D051
:1064300005481D30FCF782FD0020207000F00CF8AC
:10644000284670BD0C0A0020CC000C00014890F8D2
:10645000800070470C0A00202DE9F041104C207894
:1064600000281AD194F88000002816D108250126AA
:1064700000276069FCF782FF18B184F880606069CA
:1064800020616069401C6061082800D1676194F850
:106490008000002801D16D1EEBD1BDE8F081000025
:1064A0000C0A002070B5224C207810B12148FCF76E
:1064B00045FD94F880000025F8B12069606000F087
:1064C00074F8A06018B91B48C01DFCF737FDA06820
:1064D0004078C00705D194F8810010B10220E56032
:1064E00009E0606800F02BF8032806D200F012FBE8
:1064F000E06010B10120207002E02078002815D063
:10650000A06818B90B482030FCF718FD20696060BE
:1065100004EB8000C17E491CC17684F88050C27EA5
:10652000A068417862F342014170012070BD000013
:106530000C0A002098000C000830FCF7A3BE0830BD
:10654000FCF71CBF0830FCF729BF0830FCF776BF0A
:1065500001480078704700000C0A002010B504467E
:1065600000F0C4FA2046BDE81040FCF78BBEFCF7F3
:1065700005BF70B50446FCF711FF050002D02046A8
:1065800000F0B4FA284670BD70B50E4604460025EA
:10659000FCF798FE38B121463046FCF721FF10B1D8
:1065A000FFF75AFF0125284670BDFCF747BF0000E2
:1065B00001480078704700002C0100200448017851
:1065C000817041780170001D50F8210000470000E3
:1065D0002C01002002498870487008707047000044
:1065E0002C01002001484078704700002C01002059
:1065F00010B50446022802D30248FCF79FFC02486B
:10660000447010BD33000D002C01002040580028BC
:1066100000D00120704708B5002242504058009039
:1066200008BDD0F80403084000D00120704740584E
:10663000002800D00120704708B500224250405881
:10664000009008BD002802D001498001084770472A
:10665000217300000121B1EB507F01D1012070476F
:106660000020704770B50D4600F0E2FA04000FD02C
:106670000020FAF7B8FA207920B10020FAF7B5FA2D
:10668000112070BD0120256020710020FAF7ADFABD
:10669000002070BD10B500F0CBFA002802D0002118
:1066A0000160017110BD00000149024800F0ACBC5E
:1066B000E0010020002000402DE9F041054600796E
:1066C00016460F4600EB40012D4A01EBC00102EBDC
:1066D000810494F82A1011B10820BDE8F0812949FD
:1066E00051F820102868FFF7BDFF08B11120F4E72A
:1066F00039462846FAF78EFA66603869206030001D
:106700004FF001062FD03F7F4FF48E712868FFF7BE
:1067100082FF4FF4A2712868FFF77DFF28681A49AD
:10672000C0F8041328684FEA4711000B40B2002854
:1067300006DA00F00F0000F1E02080F8141D03E0FD
:1067400000F1E02080F800142868000B40B200F04F
:106750001F0206FA02F14009800000F1E020C0F8B3
:106760008012C0F8001128680421C0F8001500202C
:10677000A061E06184F8290044F8140FA675ACE725
:10678000E001002014730000800002002DE9F047B2
:10679000054600790B4600EB400101EBC0002349A0
:1067A00001EB8004284600F043F810B11120BDE849
:1067B000F0874FF00008C4F82080A360626184F87D
:1067C00028804FF48E76474631462868FFF723FF2E
:1067D00028684FF00109C0F808902146286800F0A9
:1067E000AFFB606800BBD5F800A00EE094F828006D
:1067F00008B10F2716E031465046FFF707FF002883
:10680000F4D02146504600F09BFB216A606981422A
:10681000F1D331462868FFF7F9FE0028F9D028683F
:10682000C0F80C90C4F814803846C0E7E00100209E
:10683000007900EB400101EBC000044901EB80004E
:106840004069002800D0012070470000E0010020CE
:106850002DE9F047044600794FF0000900EB4001B4
:1068600001EBC000254901EB80072068C0F80095C6
:10687000786880B120682249C0F808132068012197
:10688000000B40B200F01F0291404009800000F16F
:10689000E020C0F880112068D0F80C25D0F81485CD
:1068A000D0F80865D0F810554FF0FF31C0F8141536
:1068B000C0F80C152068C0F80815C0F81015501C59
:1068C00002D01046FDF710F8B8F1FF3F02D0404665
:1068D000FDF70AF8681C02D02846FDF705F8701C81
:1068E00002D03046FDF700F82068FFF7D3FE87F8A6
:1068F0002A90C7F80490BDE8F0870000E00100206E
:10690000840202000149024800F02ABC0C02002067
:10691000002000402DE9F0410546164600790F465B
:10692000154A00EBC00102EB810494F8201011B16C
:106930000820BDE8F081114951F820102868FFF7C0
:1069400091FE08B11120F4E739462846FAF7A6F976
:106950006660386920601EB1397F2846FBF7CAFFA0
:1069600028680821C0F800150020A061E06101211D
:10697000606184F82010DCE70C020020187300002E
:106980002DE9F04704460E460079204900EBC0008F
:1069900001EB800517463046FFF75CFE30B120461C
:1069A00000F036F820B11120BDE8F0871020FBE799
:1069B0006F61AE604FF49076002731462068FFF794
:1069C0003BFE4FF4AC7841462068FFF735FE206867
:1069D000AA686969C0F84425C0F8481520680121F3
:1069E0008160686878B9B14649462068FFF71FFEA4
:1069F000064641462068FFF71AFE0643F4D000B170
:106A00000F27002068613846CEE700000C02002006
:106A10000079054900EBC00001EB800040690028C7
:106A200000D00120704700000C0200202DE9F04743
:106A300004460079274900EBC00001EB800720687D
:106A40004FF00009C0F80095786880B120682249AD
:106A5000C0F8081320680121000B40B200F01F02AB
:106A600091404009800000F1E020C0F880112068CA
:106A7000D0F80C25D0F81485D0F80865D0F810555A
:106A80004FF0FF31C0F80C15C0F814152068C0F89D
:106A90000815C0F81015501C02D01046FCF72DFF49
:106AA000B8F1FF3F02D04046FCF727FF681C02D038
:106AB0002846FCF722FF701C02D03046FCF71DFF71
:106AC0002068FFF7E7FD87F82090C7F80490BDE83D
:106AD000F08700000C02002010030200024A00218F
:106AE00002EB8000816170470C0A002010B504465B
:106AF000064890F8801021B10069A04201D1FFF74B
:106B0000ABFC03490020085510BD00000C0A002012
:106B10002401002010B5044CE06F002802D1FCF7DE
:106B2000A9FCE06710BD00000C0A002070B5094DFB
:106B30000446E86F10B90848FCF700FA04F10801B0
:106B4000E86FFCF74DFC002802D00020E867012028
:106B500070BD00000C0A00202E020C0010B50C467F
:106B6000017A052908D0407A38B1084808A102689E
:106B70002046FCF77DFD00E01AB106A12046FCF797
:106B800077FD2046BDE81040FCF77FBD880000205F
:106B9000257300000D0A000038B5C3880D46044671
:106BA00033B114A0009015A216A12846FCF760FD91
:106BB000217A05291CD0607A48B1A088FEF7BEFF73
:106BC000164951F8202016A12846FCF751FDA0884F
:106BD0000021FFF775F903461049207A143951F85E
:106BE000202001B02846BDE830400EA1FCF740BD92
:106BF00038BD00001B5B306D000000001B5B313BAB
:106C000033316D0025734C6F67732064726F707041
:106C10006564202825642925730D0A00880000205A
:106C2000257300003C25733E2025733A20000000A8
:106C30000349884201D10348704700207047000093
:106C4000002000401800002070B5012670044FF0AD
:106C5000E0210025C1F88001084C4010C4F8480329
:106C6000C4F8080366602F20FFF7ECFCA660044C14
:106C70002F20A560FFF7E6FCA57070BD0010014055
:106C80002000002070B5054688690C4600284FF4A6
:106C9000847128460AD0FFF7BEFCD5F81805626A51
:106CA000E1688854606A401C606270BDFFF7B3FC05
:106CB000D5F8180570BD1FB501238DF80030CDE95A
:106CC0000121D0E90012684690471FBD1FB501237E
:106CD0008DF800308DF808100192D0E90012684656
:106CE00090471FBD70B50D4C0020D2B22070201D02
:106CF0000B4D0378EB5C1BB1001DFFF741FE02E07A
:106D00000C30FFF743FD08B1F9F762FF6078002807
:106D100002D021780029FAD070BD00003800002090
:106D2000000000202DE9F84F204D92468946064686
:106D30009846012269461846AF68FAF74BF858B3EF
:106D4000009800210446801C09E000BF00EA070308
:106D50005AF8212005EB8303401C491CDA604145A9
:106D6000F4D34FEA164AFAF7F1F84AEA0041601CF8
:106D7000384005EB80003C4005EB8402C160D068E0
:106D800066F3C50068F3891069F39F2020F00300C3
:106D9000401C20F00400D06095F8200402E000BF01
:106DA000FEF7F2FE0028FBD1BDE8F88F3C0400207E
:106DB0002DE9F84F1D4C00256846D4E901A6FAF7E5
:106DC000CFF8002738B30023009A61681CE0D1F89F
:106DD00000C00846944503D9ACEB02020A6015E0F6
:106DE000A2EB0C0263440760D0F80CC0C169814675
:106DF000BCF1000F08D006EB030828F07F48C0E97B
:106E0000018CC9F81C5005460029E0D12846616074
:106E1000FBF7D6FD03E02846FBF7D2FD10B1504644
:106E2000FAF73EF8E770BDE8F88F00002000002078
:106E30000D4B10B5596831B102680C68A24204D8F4
:106E4000A21A0A60C161586010BD0B4603E00B46F0
:106E5000C969121B21B10C689442F8D3A41A0C60C2
:106E60000260C161D86110BD200000202DE9F04111
:106E7000144E77683D462C4603E0844204D02546F4
:106E8000E469002CF9D11BE0D4B1A5420BD1F8691B
:106E9000706040B90C49012088600021B160F07039
:106EA0002F20FFF7CFFB2168E069E86110B102688D
:106EB000114401607068874202D00120BDE8F08172
:106EC0000020FBE720000020001001402DE9F041E8
:106ED000194D6C68002C2CD0184800270068A96850
:106EE000B846401A20F07F462068B0420CD82146B0
:106EF000361A0744E469087C20B181F8108088695B
:106F000049698847002CEFD129786878814206D1F9
:106F1000401CC0B26870022801D185F80180064883
:106F200069780C3040F82170BDE8F0411420F9F781
:106F300060BBBDE8F0810000200000200415014086
:106F400070B50C4605464FF48E71FFF764FB216A5D
:106F5000A068415C206A401C2062C5F81C1570BD09
:106F60001FB500228DF800200291816801914261D5
:106F7000D0E90012684690471FBD00001FB50A46C1
:106F800001788DF8001041680191017A8DF80810A0
:106F9000C0680390044850F82210001F50F82220C7
:106FA000684690471FBD00000800002001490120ED
:106FB000087070473800002010B588B004462022C1
:106FC0000E496846F9F7AEF906200090C01F0190FF
:106FD000029003904FF0EB7006900CB1084A00E06D
:106FE000002269460748FCF7D5F808B1F9F7F0FD2B
:106FF0000448001F447008B010BD00004473000036
:10700000AD6F00003C0000202DE9FF470C4605460F
:107010004FF40071FFF705FB01274FF401780026BC
:1070200018B34FF4927949462846FFF7EFFAE0B1DA
:1070300049462846FFF7EFFAC5F8088394F8290077
:1070400000B96F6002208DF80000D5F88004C5F803
:1070500080040390A0690290E0680190A661E66157
:10706000D4E900126846904728E004212846FFF73B
:10707000D8FA18B34FF484712846FFF7C7FAE8B17D
:1070800021462846FFF7FEFD616AA069884215D1B6
:10709000E06938B1E268616AA0612069E661666210
:1070A000E06008E094F8290000B96F60C5F8088333
:1070B000A661E268616A2046FFF7FDFD4FF48E7815
:1070C00041462846FFF7A2FA78B1206A61698842F2
:1070D00002D294F8280020B341462846FFF79BFAD5
:1070E000616911B12046FFF73BFF4FF4A27841469A
:1070F0002846FFF78BFA002818D041462846FFF7AC
:107100008AFA94F8290000B12F60A06900280DD0F8
:10711000A661E268616A04B02046BDE8F047FFF767
:10712000CABD21462846FFF70BFFDEE7BDE8FF8713
:107130001FB50A4601788DF8001041680191017A67
:107140008DF80810C0680390044850F82210001F02
:1071500050F82220684690471FBD0000080000201C
:107160002DE9FF410C464FF4927705463946FFF76B
:107170005EFA0026C0B139462846FFF75DFA0220C4
:107180008DF80000D5F88004C5F880040390D5F888
:107190003C058DF80800E0680190A661E661D4E93D
:1071A00000126846904723E04FF488773946284616
:1071B000FFF73DFAE0B139462846FFF73DFAD5F82A
:1071C0003C15A069884213D1E06960B1E268D5F846
:1071D000000220F02000C5F80002E069A0612069EB
:1071E000E661E06001E0A661E2682046FFF76EFD1F
:1071F0004FF4A27739462846FFF719FA60B13946AD
:107200002846FFF719FAA06930B1A661D5F83C15F8
:107210002046E268FFF75AFD4FF49077394628463A
:10722000FFF705FA002813D039462846FFF704FA7D
:10723000606900280CD0D5F84C058DF800608DF8F9
:107240000800A06801906661D4E900126846904782
:10725000BDE8FF812DE9F05F8346DDE90A4A9946E2
:1072600090460D460846012703E000BFB0FBF8F04A
:107270007F1C4045FAD2B94500D94F465FEACA7033
:1072800012D18CB15FEA8A7002D5B9F1000F01D03A
:10729000202607E0302605E031465846641EF9F7FF
:1072A000DDFD0CB1A742F7D35FF00106B9F1010F84
:1072B00002D9A9F1010903E0B5FBF6F0404502D37C
:1072C00006FB08F6F2E7DFF83C9000BFB5FBF6F0EE
:1072D00000FB165519F800105846F9F7BFFDB6FB2C
:1072E000F8F6002EF2D15FEACA7009D0002C07D060
:1072F000A74205D220215846641EF9F7AFFDF5E7F5
:10730000BDE8F09F26730000111213140D0E0F102C
:1073100000000050A96600000569000000000000A0
:107320000338FDD870473031323334353637383989
:107330004142434445460000255B0000F95A0000E5
:10734000F15A0000FFFFFFFFFFFFFFFFFFFFFFFFFE
:10735000FFFFFFFF00000000000000000000D6015A
:107360000701000032536601172D391A440C400DF5
:10737000490D3E1A2D0C4D000000000000000000D9
:107380000338FDD870470000001000401011004085
:107390000310000001000000001000400000000089
:1073A0000B02040000000000041000400000000078
:1073B0000701030100000000004040404040404001
:1073C00040404141414141404040404040404040B8
:1073D000404040404040404040050202020202025C
:1073E00002020202020202020220202020202020AB
:1073F00020202002020202020202909090909090BF
:10740000101010101010101010101010101010107C
:1074100010101010020202020202888888888888F0
:1074200008080808080808080808080808080808DC
:10743000080808080202020240000000B9730000B8
:107440007761726E696E670064656275670000003F
:107450001B5B313B33306D001B5B306D0000000067
:107460001B5B313B33316D001B5B313B33326D00B5
:107470001B5B313B33336D001B5B313B33346D00A1
:107480001B5B313B33356D001B5B313B33366D008D
:107490001B5B313B33376D00696E666F0000000087
:1074A0006572726F720000004750494F54450000EA
:1074B000505253005541525400000000554152545F
:1074C0004500000062616C6C6F632E6C6F675F6DCE
:1074D000656D706F6F6C0000617070004475000026
:1074E0000000002054010000B80300009075000067
:1074F00054010020142B0000440B0000A87400006D
:1075000000000000B074000000000000B47400002F
:1075100000000000BC74000000000000C474000003
:1075200000000003D8740000000003036400002082
:107530005C000020640000207C0300204C0100203F
:10754000180000000142642000405420004003273E
:10755000387333A074334074339874334874335899
:107560007433507433607433687433707433787464
:1075700033807433887403209074041190D003C254
:1075800005064404192A3F4D335D4B031F214B0070
:0400000500000201F4
:00000001FF
